S01900006F70656E626C745F73746D3332663230372E7372656300
S315080000000000022041070008250700082707000806
S31508000010290700082B0700082D0700080000000024
S315080000200000000000000000000000002F07000884
S3150800003031070008000000003307000835070008EC
S315080000409107000891070008910700089107000822
S315080000509107000891070008910700089107000812
S315080000609107000891070008910700089107000802
S3150800007091070008910700089107000891070008F2
S3150800008091070008910700089107000891070008E2
S3150800009091070008910700089107000891070008D2
S315080000A091070008910700089107000891070008C2
S315080000B091070008910700089107000891070008B2
S315080000C091070008910700089107000891070008A2
S315080000D09107000891070008910700089107000892
S315080000E09107000891070008910700089107000882
S315080000F09107000891070008910700089107000872
S315080001009107000891070008910700089107000861
S315080001109107000891070008910700089107000851
S315080001209107000891070008910700089107000841
S315080001309107000891070008910700089107000831
S315080001409107000891070008910700089107000821
S315080001509107000891070008910700089107000811
S315080001609107000891070008910700089107000801
S315080001709107000891070008910700080000000091
S3090800018091070008CD
S3150800018410B5054C237833B9044B13B10448AFF3BF
S3150800019400800123237010BDE00100200000000048
S315080001A4BC55000808B5034B1BB103490348AFF314
S315080001B4008008BD00000000E4010020BC550008CA
S315080001C408B502F03BFC08BD08B502F047FC08BDBB
S315080001D408B5054B1B6913F4005F01D1002008BD5F
S315080001E400F0D2F80120FAE70008024008B56420B6
S315080001F400F09AF808BD08B500F09CF808BD0000A0
S3150800020400B5C7B04FF48C720021684605F0BEF9F4
S315080002146946094805F032F840B9009B53B19DF880
S31508000224083013F0100F02D1012000E0002047B077
S315080002345DF804FB0020FAE7E45500080048704717
S31508000244E455000808B50748002380F828320A222E
S31508000254054904F079FC18B9024B012283F82822CF
S3150800026408BD00BFFC010020D455000810B50D4B8D
S3150800027493F82832012B10D002F08CFB00F16404A9
S31508000284094B1B6813F0400F03D102F083FBA0420D
S31508000294F6D9064805F01CF810BD024804F020FFFC
S315080002A4EAE700BFFC01002000480040E4550008C6
S315080002B408B5054B93F82832012B00D008BD02482F
S315080002C404F00EFFFAE700BFFC01002038B5054626
S315080002D4134B93F82832012B0CD1114905F080F8F9
S315080002E4002807DA0E48002380F8283204F0F8FEBE
S315080002F400E001352B788BB10A4A536002F04AFBB9
S3150800030400F10A04074B1B6813F0800FF1D102F0C1
S3150800031435FC02F03FFBA042F4D9EAE738BD00BF3A
S31508000324FC01002000480040014B1880704700BFBC
S315080003342804002008B502F02DFB0F4B1B689842D1
S3150800034410D30E4B1B7873B90C4B01221A700C4B45
S315080003544FF480729A6102F01DFB0A4B1B881844FD
S31508000364054B186008BD054B00221A70044B4FF064
S3150800037480729A61EFE700BF2C0400202A0400204B
S315080003840014024028040020024B4FF080729A6140
S31508000394704700BF001402402DE9F0418CB00024D8
S315080003A40794089409940A940B942D4B1A6B42F0FB
S315080003B404021A631A6B02F004020592059A1A6B70
S315080003C442F020021A631A6B02F020020492049A7D
S315080003D41A6B42F080021A631A6B02F080020392C7
S315080003E4039A1A6B42F008021A631A6B02F008029F
S315080003F40292029A1A6B42F002021A631B6B03F00A
S3150800040402030193019BDFF864804FF08073C8F8F8
S315080004141830144F4FF48023BB610CAD4FF40053CE
S3150800042445F8183D2946104801F05EF84FF48073E4
S31508000434069301260796089409940A96294640467F
S3150800044401F052F8042306930796032308930994A4
S315080004540A942946384601F047F80CB0BDE8F081FD
S3150800046400380240000C0240000802400014024012
S315080004742DE9F04190B0002409940A940B940C9445
S315080004840D940E940F9406940794274B1A6C42F411
S3150800049480221A641A6C02F480220292029A1A6B57
S315080004A442F008021A631B6B03F008030193019BCD
S315080004B44FF4807303934FF00208CDF81080032796
S315080004C4059707260896194D03A9284601F00CF83E
S315080004D44FF400730393CDF8108005970694079498
S315080004E4089603A9284600F0FFFF4FF4E133099361
S315080004F40A940B940C940C230D930E940F940C4CA1
S3150800050409A9204601F062F9236923F4904323617B
S31508000514636923F02A036361E36843F40053E360E1
S3150800052410B0BDE8F08100BF00380240000C02405C
S315080005340048004008B5254A136823F00F0343F022
S3150800054403031360214B1B6803F00F03032BF9D134
S315080005541F4A136843F4803313601D4B1B6813F456
S31508000564003FFAD01A4B5A681A4911401A4A0A43E4
S315080005745A601A6842F080721A60154B1B6813F0A9
S31508000584007FFAD0124B9A6822F0F0029A609A68B1
S3150800059422F4E05242F4A0529A609A6822F4604225
S315080005A442F400429A609A6822F0030242F0020278
S315080005B49A60074B9B6803F00C03082BF9D107488C
S315080005C401F0A8F9002000F0F9F808BD003C024043
S315080005D4003802400080BCFF193C4000000E270783
S315080005E408B500F011F9FFF7A5FFFFF7D5FEFFF7E9
S315080005F43FFFFFF7E5FDFFF7E7FDFCE782B00021C3
S3150800060400910B4B5A6C42F480425A645A6C02F4B9
S3150800061480420092009A01911A6C42F080521A6440
S315080006241B6C03F080530193019B02B0704700BF13
S315080006340038024000B589B0002303930493059358
S31508000644069307930268154B9A4202D009B05DF8DF
S3150800065404FB0021019103F5EA331A6C42F0007297
S315080006641A641A6C02F000720192019A02911A6BCA
S3150800067442F002021A631B6B03F002030293029B05
S315080006844FF4407303930223049303230693092325
S31508000694079303A9024800F0A5FDD7E700640040C4
S315080006A40004024008B500F0B7FF18484FF08073FD
S315080006B4836100F07DFE164800F07AFE154800F0C6
S315080006C477FE154800F074FE144B1A6C22F000727B
S315080006D41A641A6C22F480221A641A6B22F0200215
S315080006E41A631A6B22F008021A631A6B22F00402C0
S315080006F41A631A6B22F002021A631A6C22F08052E9
S315080007041A645A6C22F480425A6408BD00140240E2
S31508000714000C02400008024000040240003802406F
S315080007247047FEE7FEE7FEE7FEE770477047704747
S3150800073408B500F083F808BD70470000DFF834D028
S31508000744002103E00C4B5B58435004310B480C4B17
S3150800075442189A42F6D30B4A02E0002342F8043BB5
S31508000764094B9A42F9D3FFF7E7FF04F0CBFEFFF7EC
S3150800077437FF7047000002204C5E00080000002086
S31508000784E0010020E00100209C110020FEE70000A3
S3150800079410B5094B4FF0FF321A6200241C625A62E4
S315080007A45C621A611C615A615C619A619C61FFF71B
S315080007B479FF204610BD00BF0038024010B5044634
S315080007C40E4B18784FF47A73B3FBF0F30C4A10689F
S315080007D4B0FBF3F000F010FB68B90F2C01D9012027
S315080007E40AE0002221464FF0FF3000F0D1FA054B0B
S315080007F41C60002000E0012010BD00BF040000209A
S31508000804000000200800002008B50B4B1A6842F4C3
S3150800081400721A601A6842F480621A601A6842F40E
S3150800082480721A60032000F0A1FA0020FFF7C6FFC1
S31508000834FFF7E4FE002008BD003C0240034A1168A5
S31508000844034B1B780B441360704700BF78110020D4
S3150800085404000020002800F0A18038B5044690F86A
S315080008642030D3B12268136823F00203136002F020
S3150800087499F8054623685A6812F0020F10D002F058
S3150800088491F8401B0A28F5D9636A43F40033636276
S31508000894052384F82030012038BDFFF7CBFEE1E7B5
S315080008A41A6842F001021A6002F07CF805462368C9
S315080008B45A6812F0010F0DD102F074F8401B0A2889
S315080008C4F5D9636A43F400336362052384F8203058
S315080008D40120E1E7227E012A3DD01A6822F080022F
S315080008E41A60637E012B3BD02268136823F0400309
S315080008F41360A37E012B39D02268136823F02003E2
S315080009041360E37E012B37D02268136843F0100383
S315080009141360237F012B35D02268136823F008035C
S315080009241360637F012B33D02268136823F0040312
S315080009341360A368E2681343226913436269134385
S315080009446268013A21681343CB610020606201237F
S3150800095484F82030A0E71A6842F080021A60C0E7DB
S315080009642268136843F040031360C2E722681368D9
S3150800097443F020031360C4E72268136823F01003C6
S315080009841360C6E72268136843F008031360C8E7D0
S315080009942268136843F004031360CAE7012070470A
S315080009A490F82030013BDBB2012B05D9436A43F4A6
S315080009B4802343620120704770B4434BD3F8002266
S315080009C442F00102C3F80022D3F8002222F47C5232
S315080009D4C3F80022D3F80022486A42EA0022C3F880
S315080009E400224A6902F01F02012000FA02F2D3F833
S315080009F41C42D0430440C3F81C42CB69B3B9324BFA
S31508000A04D3F80C420440C3F80C42CE688D884C696E
S31508000A1445EA0645483443F834508E680C884D69CF
S31508000A2444EA0644483503EBC5035C60CB69012BED
S31508000A341DD08B69002B32D1234CD4F804320340E1
S31508000A44C4F804320B698BBB1F4BD3F814422040FD
S31508000A54C3F814020B6A012B2FD01B4AD2F80032B2
S31508000A6423F00103C2F80032002070BC7047164B0D
S31508000A74D3F80C421443C3F80C420E688D884C69AB
S31508000A8445EA0645483443F834508E688C894D69DE
S31508000A9444EA0644483503EBC5035C60C9E70A4CD7
S31508000AA4D4F804321343C4F80432CBE70648D0F822
S31508000AB414321343C0F81432CCE70349D1F81C3274
S31508000AC41A43C1F81C22C8E70064004038B590F8F8
S31508000AD42030DBB2012B05D0436A43F4002343627A
S31508000AE4012038BD0446022380F8203002681368C2
S31508000AF423F00103136001F055FF054623685B687C
S31508000B0413F0010F0DD001F04DFF401B0A28F5D94B
S31508000B14636A43F400336362052384F820300120B2
S31508000B24DFE700206062DCE770B490F820400568CF
S31508000B34AD68013CE4B2012C06D9436A43F4802328
S31508000B444362012070BC704715F0E05F5BD0C5F3C3
S31508000B540165022D3ED80124AC401C608B68002B2D
S31508000B643ED10E68CB68046843EA465605F1180375
S31508000B741B01E65003680C6905F1180603EB061316
S31508000B845C600B7D012B36D0D17993791B0443EA3B
S31508000B940163517943EA01231479016823432C013B
S31508000BA42144C1F88C31D17893781B0443EA016354
S31508000BB4517843EA0123117802680B432244C2F8A8
S31508000BC48831026818352D01535943F001035351EE
S31508000BD40020B7E7436A43F4000343620120B1E700
S31508000BE44C6843EAC403CC680668234305F1180431
S31508000BF424013351BEE7036803EB0613596841F42D
S31508000C0480715960C0E7436A43F4001343620120C4
S31508000C1498E790F82030013BDBB2012B01D900207C
S31508000C24704703689B68890631EA030301D00120EB
S31508000C3470470020704730B490F82040013CE4B275
S31508000C44012C06D9436A43F480234362012030BC4D
S31508000C54704700296FD10468E46814F0030F64D060
S31508000C64056801F11B0424012C5904F0040494605A
S31508000C74002C6BD1056801F11B0424012C59640D61
S31508000C841460056801F11B0424012D5905F00205B9
S31508000C94D560056825446D6805F00F051561056876
S31508000CA425446D68C5F30725956105682C44646871
S31508000CB4240C546104680A011444D4F8B8411C701D
S31508000CC404681444D4F8B841C4F307245C7004686F
S31508000CD41444D4F8B841C4F307449C700468144413
S31508000CE4D4F8B841240EDC7004681444D4F8BC4122
S31508000CF41C7104681444D4F8BC41C4F307245C7119
S31508000D0404681444D4F8BC41C4F307449C710468C9
S31508000D142244D2F8BC21120EDA71F9B90268D368F2
S31508000D2443F02003D360002091E7436A43F4001399
S31508000D34436201208BE70468246914F0030F8FD1FA
S31508000D44436A43F400134362012080E7056801F10E
S31508000D541B0424012C59E408546092E702681369B9
S31508000D6443F020031361002071E70000074AD368A3
S31508000D7423F4E0631B041B0C000200F4E060184330
S31508000D8440F0BF6040F40030D060704700ED00E0EA
S31508000D9430B4174BDB68C3F30223C3F10704042CEE
S31508000DA428BF04241D1D062D18D9033B4FF0FF3513
S31508000DB405FA04F421EA0401994005FA03F322EA40
S31508000DC40303194300280BDB0901C9B200F160408B
S31508000DD400F5614080F8001330BC70470023E5E74E
S31508000DE400F00F000901C9B2024B1954F4E700BF19
S31508000DF400ED00E014ED00E00138B0F1807F0AD27E
S31508000E04064B5860064AF02182F8231000209860A1
S31508000E1407221A6070470120704700BF10E000E0FF
S31508000E2400ED00E010B409490C6924F440740C611F
S31508000E340C6944F440740C610C6944F001040C61B7
S31508000E440260BFF36F8F436010BC7047003C0240DA
S31508000E54074B1A6922F440721A611A6942F400723D
S31508000E641A611A6942F001021A610160704700BFEB
S31508000E74003C0240074B1A6922F440721A611A6947
S31508000E8442F480721A611A6942F001021A610180F9
S31508000E94704700BF003C0240064B1A6922F44072B0
S31508000EA41A611A691A611A6942F001021A61017013
S31508000EB4704700BF003C0240204BDB6813F0100F5C
S31508000EC407D01F4AD36943F00803D3611B4B10228A
S31508000ED4DA601A4BDB6813F0200F07D0184AD36977
S31508000EE443F00403D361154B2022DA60134BDB6805
S31508000EF413F0400F07D0124AD36943F00203D361B3
S31508000F040E4B4022DA600D4BDB6813F0800F07D0D6
S31508000F140B4AD36943F00103D361084B8022DA6094
S31508000F24064BDB6813F0020F07D0054AD36943F072
S31508000F341003D361014B0222DA607047003C024079
S31508000F447C110020094B1B69002B01DB002070472C
S31508000F54064B074A5A6002F188325A601B69002B0D
S31508000F6401DB002070470120704700BF003C0240A7
S31508000F7423016745034A136943F0004313610020BC
S31508000F84704700BF003C024038B50446154B0022A2
S31508000F94DA6101F007FD0546134BDB6813F4803F5D
S31508000FA40AD0B4F1FF3FF7D0CCB101F0FBFC401BEB
S31508000FB4A042F1D903200DE00B4BDB6813F0010FB7
S31508000FC402D0094B0122DA60074BDB6813F0F20FF3
S31508000FD401D1002038BDFFF76FFF0120FAE703208F
S31508000FE4F8E700BF7C110020003C0240F8B51D4C10
S31508000FF4247E012C34D01F4616460D460446194B4A
S3150800100401221A764CF25030FFF7BEFF014698B912
S31508001014BCB1012C1AD0022C1DD032463B462846B8
S31508001024FFF700FF4CF25030FFF7AEFF01460E4AB9
S31508001034136923F0010313610A4B00221A76084642
S31508001044F8BDF1B22846FFF727FFEBE7B1B2284609
S31508001054FFF710FFE6E731462846FFF7F9FEE1E712
S315080010640221ECE77C110020003C0240074B1A6978
S3150800107422F440721A611A6942F004021A611A6962
S3150800108442EA002040F4803018617047003C024070
S3150800109410B449B1012925D0022902D04FF440746D
S315080010A403E04FF4007400E00024104B196921F49E
S315080010B4407119611A6922431A611A6922F0F80201
S315080010C41A61F82292FAA2F2B2FA82F2904040F039
S315080010D402001A69104318611A6942F480321A61C7
S315080010E410BC70474FF48074DFE700BF003C024031
S315080010F4164B1B6813F4007F10D0144B1A6822F49D
S3150800110400721A601A6842F400621A601A6822F4B5
S3150800111400621A601A6842F400721A600B4B1B6864
S3150800112413F4806F10D0094B1A6822F480621A608F
S315080011341A6842F480521A601A6822F480521A60B5
S315080011441A6842F480621A60704700BF003C024085
S31508001154F8B5224B1B7E012B3ED00E4604461F4B88
S3150800116401221A764CF25030FFF70EFF074670BB81
S315080011744FF0FF3333602368012B16D0A568E36864
S31508001184A2681344AB4220D9217C2846FFF780FF86
S315080011944CF25030FFF7F8FE114A136923F0FA03AC
S315080011A41361074680B90135E9E76168207CFFF7D2
S315080011B45DFF4CF25030FFF7E7FE0746084A13690D
S315080011C423F00403136100E03560FFF791FF034B36
S315080011D400221A763846F8BD0227FBE77C11002060
S315080011E4003C0240F0B583B0002336E0082400E052
S315080011F40024B4403C430235694E46F82540694C00
S315080012042568D44304EA05064F6817F4803F01D0DD
S3150800121442EA0506634D2E606D6804EA05064F68C2
S3150800122417F4003F01D042EA05065E4D6E60AD68CC
S3150800123404EA05064F6817F4801F01D042EA05063A
S31508001244584DAE60ED682C404E6816F4001F01D068
S3150800125442EA0504534AD46001330A6832FA03F4AD
S3150800126400F09B8001249C402240F5D04D686E1EF8
S31508001274012E03D9112D01D0122D12D186685F00D3
S315080012840325BD4026EA0506CD68BD40354385607D
S31508001294466826EA04064D68C5F300149C403443A0
S315080012A44460C5685F000324BC40E44325408E6857
S315080012B4BE402E43C6604D68022D01D0122D13D1AF
S315080012C4DE08083650F826E003F007054FEA850CD1
S315080012D40F2505FA0CF52EEA050E0D6905FA0CF527
S315080012E445EA0E0540F8265005682C404D6805F079
S315080012F40305BD402C4304604C6814F0805FABD0F2
S3150800130400240194284C656C45F480456564646C36
S3150800131404F480440194019C9D08AE1C204C54F8A6
S31508001324267003F00304A6000F24B44027EA040732
S315080013341E4CA0423FF45CAF04F58064A0421ED064
S3150800134404F58064A0421CD004F58064A0421AD037
S3150800135404F58064A04218D004F58064A04216D02F
S3150800136404F58064A04214D004F58064A04212D027
S3150800137404F58064A0423FF439AF092439E701240F
S3150800138437E7022435E7032433E7042431E7052441
S315080013942FE706242DE707242BE703B0F0BD00BF8B
S315080013A400380140003C0140003802400000024079
S315080013B4444B984219D0444B984222D0434B984206
S315080013C42BD0434B984234D0424B98423DD0424BA3
S315080013D4984246D0414B98424FD0414B984258D0F8
S315080013E4404B984261D00120704703F560531A694F
S315080013F442F001021A611A6922F001021A610020F8
S31508001404704703F550531A6942F002021A611A69C1
S3150800141422F002021A610020704703F540531A6944
S3150800142442F004021A611A6922F004021A610020C1
S31508001434704703F530531A6942F008021A611A69AB
S3150800144422F008021A610020704703F520531A692E
S3150800145442F010021A611A6922F010021A61002079
S31508001464704703F510531A6942F020021A611A6983
S3150800147422F020021A610020704703F500531A6906
S3150800148442F040021A611A6922F040021A610020E9
S31508001494704703F5E0531A6942F080021A611A6923
S315080014A422F080021A610020704703F5C0531A69B6
S315080014B442F480721A611A6922F480721A61002051
S315080014C4704700BF000002400004024000080240C2
S315080014D4000C0240001002400014024000180240AA
S315080014E4001C024000200240F0B40A6892FAA2F2F4
S315080014F4B2FA82F22DE00E69C46893FAA3F5B5FA36
S3150800150485F56D00032707FA05F524EA050493FA19
S31508001514A3F5B5FA85F56D0006FA05F52C43C460FE
S315080015244C68022C40D04C68056893FAA3F6B6FAC0
S3150800153486F67600032707FA06F625EA060593FAD9
S31508001544A3F3B3FA83F35B0004FA03F32B430360B0
S3150800155401320B6833FA02F45AD00124944023402A
S31508001564F6D04C68013C012CC5D88E68846893FA79
S31508001574A3F5B5FA85F56D00032707FA05F524EAF8
S31508001584050493FAA3F5B5FA85F56D0006FA05F58B
S315080015942C4384600E68CD68446824EA060405FB77
S315080015A406F52C434460A6E793FAA3F4B4FA84F444
S315080015B4072C15D84E69046A93FAA3F5B5FA85F586
S315080015C4AD000F2707FA05F524EA050493FAA3F5EF
S315080015D4B5FA85F5AD0006FA05F52C430462A2E7CB
S315080015E44D69466A1C0A94FAA4F7B7FA87F7BF0046
S315080015F44FF00F0C0CFA07F726EA070694FAA4F438
S31508001604B4FA84F4A40005FA04F4344344628AE779
S315080016140020F0BC70470000154A136843F0010324
S315080016241360134B1B6813F0020FFAD0104A0023F9
S315080016349360104B1360136823F0F80343F0800398
S3150800164413600B4B1B6813F0007FFAD1084B1B6819
S3150800165413F0006FFAD1064B074A5A60074AC3F8D3
S3150800166484200020D8605A6F42F080725A67704707
S3150800167400380240FFFFF2FA103000240030002040
S31508001684034B9B68C3F30313024AD35CD8407047E1
S315080016940038024000560008034B9B68C3F38223B4
S315080016A4024AD35CD84070470038024010560008F6
S315080016B4034B9B68C3F34233024AD35CD840704752
S315080016C400380240105600080D4B5B6803F480038B
S315080016D40BB90C4800E00C48094A536803F03F0369
S315080016E4B0FBF3F35068C0F3881000FB03F05368AB
S315080016F4C3F3014301335B00B0FBF3F0704700BF4B
S31508001704003802400024F40040787D0108B5074BF0
S315080017149B6803F00C03042B06D0082B01D004485D
S3150800172408BDFFF7D1FFFBE70248F9E70038024096
S315080017340024F40040787D0110B50446FFF7E6FF5F
S315080017442060FFF79DFF6060FFF7A6FFA060606852
S31508001754FFF7AEFFE06010BD0246036813F0400FC2
S315080017642DD110B4006820F47F4020F0BF000B6828
S315080017744C6823438C682343CC6823430C6923436E
S315080017844C6923438C692343CC6923430C6A23435A
S3150800179403431360536823F00403C88A034353605E
S315080017A40B6AB3F5005F06D00020D36923F40063FF
S315080017B4D36110BC70478B8C13610020F5E70120B8
S315080017C4D36923F40063D36170470000C36813F434
S315080017D4005F01D00120704730B585B00D46044638
S315080017E4C36823F4164323F00C034A68C9680A43FA
S315080017F429690A43A9690A431343C360AB680269A2
S3150800180422F44052134303616B69426922F440721D
S31508001814134343616846FFF78FFF374B9C4210D04A
S31508001824364B9C4214D0364B9C4213D0354B9C42C3
S3150800183412D0354B9C4211D0344B9C4210D0012017
S3150800184458E0039B002B54D02A685AB9012051E06A
S31508001854029BF7E7029BF5E7039BF3E7029BF1E795
S31508001864029BEFE7A969B1F5004F20D003EB830388
S3150800187403EB83039200B3FBF2F3254DA5FB032088
S315080018844009020191B2642202FB10321301323379
S31508001894A5FB0323C3F34F1303F0F0020A4492B2E1
S315080018A403F00F0313449BB2A360002022E003EB6A
S315080018B4830303EB83035200B3FBF2F3144DA5FB36
S315080018C403204009020191B2642202FB1032D300BC
S315080018D43233A5FB0323C3F34F135A0002F4F872F9
S315080018E40A4492B203F0070313449BB2A360002090
S315080018F400E0012005B030BD00100140004400405E
S315080019040048004000140140004C004000500040CC
S315080019141F85EB51014B1860704700BF000000207B
S31508001924024A137843F00103137070470C00002031
S3150800193410B50D4B187301F02DF800F132040A4B5B
S315080019449B6813F0010F07D101F018F901F022F88A
S31508001954A042F4D9012300E000231BB9024BD8683E
S31508001964C0B210BD0020FCE7003C004008B5034B9C
S3150800197404229A61FF20FFF7DBFF08BD000C024032
S3150800198410B50446FF20FFF7D3FF207010BD38B505
S3150800199401F000F800F5FA75FF20FFF7C9FF0446C1
S315080019A401F0ECF8FF2C03D000F0F4FFA842F3D3BF
S315080019B4FF2C14BF0020012038BD000010B5084BC9
S315080019C44FF480229A61FF20FFF7B2FFFFF7DFFF8B
S315080019D410B10124204610BD0446FFF7C7FFF9E7F6
S315080019E4000C024070B504460E4610F0800F2DD147
S315080019F4FFF7BCFFFFF7E2FFD0B344F04000FFF760
S31508001A0497FF300EFFF794FFC6F30740FFF790FFE2
S31508001A14C6F30720FFF78CFFF0B2FFF789FFFCB186
S31508001A240120082C1ED0FFF783FF0C2C1CD00A2497
S31508001A34FF20FFF77DFF054601F0A0F815F0800F9B
S31508001A4417D0631E13F0FF04F2D112E000F07F04EE
S31508001A5400213720FFF7C6FF0546012809D8C7E73E
S31508001A649520DEE78720DEE7FF20FFF761FFDEE744
S31508001A74FF25284670BDF8B505460E4600F08AFFD0
S31508001A8400F16407FF20FFF753FF044601F076F8D8
S31508001A94FF2C03D100F07EFFB842F3D3FE2C01D00D
S31508001AA40020F8BD6C1C2846FFF76AFF204602355D
S31508001AB4FFF766FF01F062F8023EF3D1FF20FFF755
S31508001AC437FFFF20FFF734FF0120EAE770B5054624
S31508001AD40C46FFF75CFF034608B9184670BD204656
S31508001AE4FFF726FFFD2C1DD04FF400762C4614F87C
S31508001AF4020BFFF71DFF6878FFF71AFF01F03EF89F
S31508001B042546023EF2D1FF20FFF712FFFF20FFF71A
S31508001B140FFFFF20FFF70CFF00F01F00052803D076
S31508001B240023DAE70123D8E70123D6E770B586B0A0
S31508001B34234B04229A614FF480560096012301939D
S31508001B44022302930025039504951E4C69462046F4
S31508001B54FFF7CAFCA66100E00135092D1DD800F07F
S31508001B6419FF00F16404184B9B6813F0020F03D1A4
S31508001B7400F010FFA042F6D9134BFF221A7300F0A7
S31508001B8409FF00F16404104B9B6813F0010FE3D1BD
S31508001B9400F000FFA042F6D9DEE74FF48053009325
S31508001BA40223019303230293002303930493062336
S31508001BB4059369460348FFF797FC06B070BD00BF56
S31508001BC4000C024000080240003C0040F0B595B005
S31508001BD42C4B1A6B42F004021A631A6B02F00402C5
S31508001BE40392039A1A6B42F008021A631A6B02F0FC
S31508001BF408020292029A1A6C42F400421A641B6C96
S31508001C0403F400430193019B0427049701230593D6
S31508001C14022506950024079408941B4E04A9304609
S31508001C24FFF762FCB7614FF4E05304930595032369
S31508001C340693079408940623099304A91348FFF7FF
S31508001C4453FC0A944FF482730B930C940D940E94DC
S31508001C544FF400730F9330231093119412940723AF
S31508001C6413930B4C0AA92046FFF776FD636823F005
S31508001C7410036360236843F040032360FFF756FFAD
S31508001C8415B0F0BD00380240000C024000080240BE
S31508001C94003C004010B58AB0114C236823F0400379
S31508001CA42360002300934FF48272019202930393F4
S31508001CB404934FF400720592069307930893072337
S31508001CC4099369462046FFF747FD636823F0100326
S31508001CD46360236843F0400323600AB010BD00BF65
S31508001CE4003C0040002840F09C80F0B583B00446D0
S31508001CF44D4B1B7813F0020F04D04B4B1878C0B227
S31508001D0403B0F0BDFFF762FF484B4FF480229A6197
S31508001D1400210846FFF766FE0546012810D0444B05
S31508001D241C60FFF723FE002C78D03F4A137803F093
S31508001D34FE031370FFF7AEFF3B4B1878C0B2DFE71C
S31508001D4400F028FE00F57A764FF4D5710820FFF7DF
S31508001D5449FE01283CD1254608E0FF20FFF7E8FDA7
S31508001D6402AB2B4403F8040C0135EDB2032DF4D968
S31508001D749DF80630012BD2D19DF80730AA2BCED177
S31508001D8400F008FEB04206D24FF08041A920FFF7C2
S31508001D9429FE0028F4D100F0FDFDB042BFD200218F
S31508001DA43A20FFF71FFE054648B1B8E7FF20FFF7BC
S31508001DB4BFFD02AB2B4403F8040C0135EDB2032D29
S31508001DC4F4D99DF8043013F0400F25D00C24A6E767
S31508001DD40021A920FFF706FE01281AD92F4601E09B
S31508001DE400F0CCFE00F0D6FDB04205D2002128460C
S31508001DF4FFF7F8FD0028F3D100F0CCFDB0428ED2EF
S31508001E044FF400711020FFF7EDFD002887D13C46FA
S31508001E1485E70227A925E5E7042480E7FFF780FD7F
S31508001E248AE70120704700BF0C000020000C02401E
S31508001E343004002018B9034B1878C0B27047012043
S31508001E44704700BF0C00002000283BD138B50D466A
S31508001E541C46002B38D01E4B1B7813F0010F35D1C6
S31508001E641C4B1B6813F0080F00D15202012C1AD020
S31508001E7411461220FFF7B6FD78B94FF400712846CB
S31508001E84FFF7F9FD28B105F5007500F077FE013C6A
S31508001E94F3D100210C20FFF7A5FDFFF767FD201CF1
S31508001EA418BF012038BD11461120FFF79BFD0028F5
S31508001EB4F3D14FF400712846FFF7DDFD0028ECD076
S31508001EC40024EAE7042070470420EBE70320E9E747
S31508001ED40C0000203004002000284AD170B50D46B5
S31508001EE416461C46002B46D0264B1B7813F0010FCA
S31508001EF443D1244B1B7813F0040F40D1224B1B68A3
S31508001F0413F0080F00D15602012C1DD013F0060F4A
S31508001F1428D131461920FFF765FD78B9FC212846F2
S31508001F24FFF7D4FD28B105F5007500F027FE013C3E
S31508001F34F4D1FD210020FFF7C9FDC0B1FFF716FD56
S31508001F44201C18BF012070BD31461820FFF74AFD32
S31508001F540028F3D1FE212846FFF7B8FD0028EDD066
S31508001F640024EBE721469720FFF73CFDD1E701243F
S31508001F74E4E7042070470420E5E70320E3E70220AA
S31508001F84E1E700BF0C0000203004002030B585B01E
S31508001F94002840F02381934B1B7813F0010F40F07F
S31508001FA41F8114460E2900F20B81DFE811F00F0099
S31508001FB4160009015B000901090109010901090162
S31508001FC40901B700C000CF00DD00F100FFF7F6FCF9
S31508001FD4002840F0F7800124A4E000210920FFF737
S31508001FE401FD08B101249DE010216846FFF743FD71
S31508001FF4002800F0E9809DF800309B09012B20D0C9
S315080020049DF8052002F00F029DF80A3002EBD31260
S315080020149DF809305B0003F006031A449DF808107E
S315080020249DF807309B0003EB91139DF8061089026F
S3150800203401F440610B440133073A934023600024BA
S3150800204470E09DF809309DF8082003EB02239DF8FB
S315080020540720120402F47C12134401339B02236002
S3150800206400245FE0604B1B6813F0040F21D00021A5
S315080020748D20FFF7B7FC08B1012453E0FF20FFF7D2
S3150800208457FC10216846FFF7F6FC80B9012449E09D
S31508002094FF20FFF74DFC013DEDB2002DF8D19DF868
S315080020A40A301A0910239340236000243AE03025A5
S315080020B4F3E700210920FFF795FC08B1012431E074
S315080020C410216846FFF7D7FC00287FD0464B1B68CB
S315080020D413F0020F11D09DF80A305B0003F07E035B
S315080020E49DF80B2003EBD21301339DF80D209209BA
S315080020F4013A93402360002414E09DF80A30C3F3A0
S3150800210484029DF80B10CB0003F0180303EB51135C
S31508002114013302FB03332360002403E0324B1B68BC
S3150800212413700024FFF722FC204605B030BD0021B9
S315080021340920FFF757FC08B10124F3E710212046CC
S31508002144FFF799FC002843D10124EBE700210A2074
S31508002154FFF748FC08B10124E4E710212046FFF7FD
S315080021648AFCB8BB0124DDE700213A20FFF73AFCD4
S31508002174054648B10124D5E7FF20FFF7D9FB60558A
S3150800218400F0FCFC0135EDB2032DF5D90024C9E7AE
S31508002194154B1B6813F0040F01D10124C2E7002173
S315080021A48D20FFF71FFC08B10124BBE7FF20FFF7CA
S315080021B4BFFB40212046FFF75EFC68B90124B1E75E
S315080021C40424AFE70024ADE70124ABE70124A9E71B
S315080021D40024A7E70024A5E70024A3E70424A3E72B
S315080021E40324A1E70C0000203004002072B67047CF
S315080021F462B670472DE9F04184B004460D46174689
S3150800220498466846FFF798FA0299164BA3FB0131DC
S315080022148909002201E00132D2B2112A1DD8124BD3
S3150800222413F8120003EB420393F801C000EB0C0306
S3150800223403FB0443B1FBF3FE03FB1E16002EEAD18F
S315080022441FFA8EF32B80013B9BB2B3F5806FE2D263
S31508002254387088F800C0012000E0002004B0BDE80A
S31508002264F08100BFD34D62105456000870B58CB087
S315080022740022ADF82E208DF82D200CAB03F8042D82
S315080022840DF12D020DF12E014FF4FA70FFF7B2FF8E
S31508002294002835D01D4C1E4B23600025257665760F
S315080022A4A5760126E67625776577A560E5609DF827
S315080022B42D30013B1B0423619DF82C30013B1B0583
S315080022C46361BDF82E3063602046FEF7C3FA0695AF
S315080022D4079508964CF6E043019302954FF6E0738A
S315080022E4039304230493059509960E230A9301A9D7
S315080022F42046FEF755FB2046FEF7E8FB0CB070BDFA
S31508002304B521044800F052FBC4E700BF340400209A
S31508002314006400401856000810B588B040F2E1730E
S315080023240293002304930593069101AB024602A97E
S315080023340B48FEF7F9FB08B108B010BD00F02AFBFC
S3150800234400F1320401990648FEF763FC0028F3D02D
S3150800235400F014FC00F01EFBA042F3D9ECE700BF22
S315080023643404002010B588B00C46034601AA00219F
S315080023740A48FEF760FC60B9019A40F267639A421C
S3150800238401D0002006E0039B33B9059B2370012086
S3150800239400E0002008B010BD0020FBE7340400204C
S315080023A408B5FFF723FF08BD10B500F001FA00B918
S315080023B410BDFDF70DFF0028FAD000F095FBFEF7D7
S315080023C4E7F900F0BDFA00F0F7F920F0604020F0D4
S315080023D47F00044B986000F0EFF94468FFF708FFA4
S315080023E4A047E5E700ED00E070B508E04D1C461C83
S315080023F40B78037000F0C2FB304629462246531E6A
S315080024049CB2002AF2D170BD38B50546002401E015
S315080024140134E4B2052C15D800F0B0FB04EB4402F1
S315080024249300094AD358AB42F2D804EB440291000C
S31508002434054A0A4452681344AB42E9D9024B0B4491
S31508002444187A00E0FF2038BD7856000808B5C1F3AD
S31508002454080353B903688B4209D040F8041B4FF4A8
S315080024640072FFF7C1FF012000E0002008BD01202B
S31508002474FCE72DE9F0410746FEF764FD00247F2CAE
S3150800248414D83E68A30006EB03083B445D6800F0D5
S3150800249475FB2A46002341460220FEF7A7FD38B9F4
S315080024A456F82430AB4209D10134E8E7012400E0A8
S315080024B40024FEF75FFD2046BDE8F0810024F8E716
S315080024C438B50D460C4B984211D004460B4B99422D
S315080024D407D1094C29462046FFF7B8FF48B12046DC
S315080024E438BDFFF7C6FF0028F4D10024F7E7044CEB
S315080024F4F0E70024F3E700BF600600200080000828
S315080025045C0400202DE9F04106460C4617461D4694
S3150800251421F4FF7828F001080368B3F1FF3F07D0D8
S31508002524336843450BD13368E41A3444043415E05C
S315080025344146FFF78BFF03460028F1D11FE04146C9
S315080025443046FFF7BDFF06460028ECD1002316E007
S3150800255417F8013B04F8013B013D0FD000F00EFBD0
S31508002564331DE31AB3F5007FF2D308F5007130463C
S31508002574FFF7A6FF064628B1041DE9E70123184616
S31508002584BDE8F0810023FAE770B586B004460D4627
S315080025940023009388420ED80126012C1ED9072D44
S315080025A420D8E6B10023019302230593012304935B
S315080025B4FEF7C8FC03E00026EFE70134E4B2AC42B8
S315080025C409D800F0DBFA0394694601A8FEF7C0FDB2
S315080025D40028F2D00026FEF7CDFC00E0002630469F
S315080025E406B070BD0026FAE74FF0FF33024A1360BF
S315080025F4024A1360704700BF5C040020600600208E
S3150800260470B54B1E154C241AA34201D9002070BD7F
S3150800261416460D460446FFF7F7FEFF281AD0281972
S315080026240138FFF7F1FEFF2816D024F4FF7323F0D0
S3150800263401030B4A934206D02B46324621460948E3
S31508002644FFF760FFE3E72B46324621460648FFF7C5
S3150800265459FFDCE70020DAE70020D8E7FFFF070880
S31508002664008000085C040020600600204A1E0E4B09
S315080026741B1A9A4201D90020704770B50C460546C4
S31508002684FFF7C2FE064660190138FFF7BDFEFF2EA6
S3150800269406D0FF2806D001463046FFF775FF70BD01
S315080026A40020FCE70020FAE7FFFF0708104B1B6829
S315080026B4B3F1FF3F1AD000B583B00D4A5368916849
S315080026C40B44D1680B4411690B4451690B44916955
S315080026D40B44D26913445B4202AA42F8043D04211E
S315080026E40448FFF78DFF03B05DF804FB012070472B
S315080026F460060020848100080D4B1B680D4A126889
S315080027041A440D4B1B6813440C4A126813440C4AAA
S3150800271412681A440B4B1B681A440B4B1B68134468
S315080027240A4A1268DA4201D000207047012070472D
S315080027340080000804800008088000080C8000084F
S315080027441080000814800008188000088481000896
S3150800275408B50D4B1B68B3F1FF3F0BD10B4B1B6838
S31508002764B3F1FF3F0DD00948FFF783FE034648B18E
S31508002774012307E00448FFF77CFE03460028EDD151
S3150800278400E00123184608BD600600205C0400200A
S31508002794004870470080000808B5FFF725FF08BD04
S315080027A408B5FFF72DFF08BD08B5FFF75FFF08BD9D
S315080027B408B5FFF7A1FF08BD08B5FFF7E9FF08BD8F
S315080027C408B5FFF773FF034608B9184608BDFFF7AF
S315080027D4BFFF0346F9E70000054B1B6813F0200FFB
S315080027E404D0034B5B6803700120704700207047D0
S315080027F40048004010B5094B586000F0CBF800F1CA
S315080028040A04064B1B6813F0800F05D100F0B6F9CD
S3150800281400F0C0F8A042F4D910BD00BF004800403B
S3150800282410B588B00C4CE36823F40053E3604FF406
S315080028346143019300230293039304930C220592A4
S315080028440693079301A92046FEF7C0FFE36843F4FD
S315080028540053E36008B010BD0048004070B5064652
S315080028640D46402904D82846FFF7C4FF00240BE088
S315080028747B21074800F09AF8F5E700F07FF9305D08
S31508002884FFF7B8FF0134A4B2ABB2A342F5D870BDC2
S31508002894C056000870B5254B1C78BCB92448FFF708
S315080028A49BFF012801D0204670BD214B1B78013BB4
S315080028B4DBB23F2BF7D800F06DF81E4B18601E4BA1
S315080028C400221A70194B01221A70ECE706460D46C7
S315080028D4194B1B78013316481844FFF77DFF044645
S315080028E4012815D1144B1A780132D2B21A70104B3A
S315080028F41B789A4201D00024D5E710493046FFF7E1
S3150800290473FD0A4B00221A700B4B1B782B70CAE70F
S3150800291400F040F8074B1B686433984203D9002437
S31508002924024B1C70BFE70024BDE700BFA5080020C2
S3150800293464080020A8080020A608002065080020CE
S31508002944024B00221A605A609A60704710E000E051
S3150800295408B5FFF7F5FF054B054A5A6000229A6049
S3150800296405211960034B1A6008BD00BF10E000E09A
S31508002974BFD40100AC080020044B1B6813F4803F45
S3150800298403D0034A136801331360704710E000E06C
S31508002994AC08002008B5FFF7EFFF014B186808BD1F
S315080029A4AC08002008B5FFF7F5FF08BD08B500F028
S315080029B4E5F8FCE708B500F0D5F8012806D000F0DC
S315080029C46BF918B10C4B1B78012B00D008BDFFF727
S315080029D4E1FF0A4B1B680A4A1268134403F5FA73A3
S315080029E49842F3D3044B00221A7000F05FF90028CA
S315080029F4ECD1FFF7D9FCE9E7B4080020B0080020B9
S31508002A04B808002008B5054B1B78012B00D008BD73
S31508002A14FFF7C0FF024B1860F9E700BFB4080020AF
S31508002A24B808002008B5044B01221A70FFF7EAFF1C
S31508002A34FFF7C0FF08BD00BFB408002008B5FFF7BC
S31508002A44AFFC00F097F8FFF783FFFFF7A5FE00F049
S31508002A540BF900F00FF8FFF7E5FF08BD08B500F01D
S31508002A648DF8FFF789FF00F01BFA00F013F8FFF75B
S31508002A74A1FF08BD10B500F095FDFFF7F7FB044C60
S31508002A8401232370FFF7CCFE0023237010BD00BF7B
S31508002A940D00002000B583B00DF107011048FFF7BB
S31508002AA461FC012809D00DF107010D48FFF7F2FE74
S31508002AB401280BD003B05DF804FB0A4B01221A70F7
S31508002AC49DF80710064800F08DFDECE7054B00223B
S31508002AD41A709DF80710024800F084FDEAE700BF63
S31508002AE4BC0800200D0000207047000038B50446D5
S31508002AF40D46094B1B78012B05D0074B1B7833B1C0
S31508002B0400F068FD38BDC9B2FFF706FCF5E7E9B27F
S31508002B142046FFF7A3FEF3E70D000020074B1B78BA
S31508002B24022B05D0032B05D0012B05D04020704776
S31508002B340020704700207047082070470D000020C9
S31508002B44074B1B78022B05D0032B05D0012B05D088
S31508002B5440207047002070470020704708207047BF
S31508002B640D00002008B500F02BFD034600B1012333
S31508002B74184608BD08B5FDF739FB08BD08B5FDF7C5
S31508002B843AFB08BD10B4034601310C4AA2FB0323E1
S31508002B94DB08F9D100230B70084BA3FB0023DB08E1
S31508002BA41A4603EB83035C00031B303301F8013D2B
S31508002BB41046002AF0D1084610BC7047CDCCCCCCC0
S31508002BC400F00F03092802D903F13700704710B53E
S31508002BD403F1300402F0BAFC2044437803F00303FB
S31508002BE4022B01D0E0B210BD203CFBE738B5054600
S31508002BF40C460009FFF7E4FF207005F00F00FFF705
S31508002C04DFFF60700023A370204638BDF8B5074679
S31508002C140026354607E0203C10E02D01EDB2AB183E
S31508002C24DDB20136F6B2012E19D8BC5D02F08EFC6F
S31508002C342044437803F00303022BECD0E3B2A3F158
S31508002C443002D2B2162A09D8A3F13A01C9B2062922
S31508002C5407D9092AE1D9373BDAB2DEE7002528463F
S31508002C64F8BD0025FBE7000008B50022064B1A70DC
S31508002C740649074801F03CFF00B908BD7721054815
S31508002C84FFF794FEF9E700BF5C0D00200057000823
S31508002C940409002004570008034B1B780BB10020D5
S31508002CA470470120704700BF5C0D002008B5FFF788
S31508002CB459FF01280ED0084B1B780BB1002008BD1C
S31508002CC4FDF79EFA012801D00020F8E7024B0122FD
S31508002CD41A70F4E70020F2E75C0D002038B50546C3
S31508002CE4047802F033FC2044437803F00303022BF0
S31508002CF403D0532C03D0032038BD203CF9E702F057
S31508002D0425FC6B781844427812F0040F09D0312B4D
S31508002D1409D0322B09D0332B01D00320ECE702204B
S31508002D24EAE70320E8E70020E6E70120E4E770B5D0
S31508002D3406460230FFF76AFF054684B20436304673
S31508002D44FFF764FF0544EDB2013CA4B20236012C38
S31508002D54F5D8ED43EDB23046FFF758FFA84201D047
S31508002D64002070BD0120FCE7F8B5044617460E4658
S31508002D74A1B198B12046FFF7B1FF0546032800F034
S31508002D8487802046FFF7D3FF002800F08480012DB2
S31508002D9429D04DB1022D4DD000257AE040F26321A9
S31508002DA43E48FFF703FEE5E7A01CFFF72FFF85B2B1
S31508002DB4201DFFF72BFF00023060A01DFFF726FF3A
S31508002DC43368184430600834033D2DB2002F60D0B0
S31508002DD40026AE425DDA2046FFF718FFB8550234DE
S31508002DE40136B6B2F5E7A01CFFF710FF85B2201D21
S31508002DF4FFF70CFF00043060A01DFFF707FF3368D8
S31508002E0403EB0020306004F10800FFF7FFFE336887
S31508002E14184430600A34043D2DB2002F39D00026F8
S31508002E24AE4236DA2046FFF7F1FEB85502340136CB
S31508002E34B6B2F5E7A01CFFF7E9FE85B2201DFFF739
S31508002E44E5FE00063060A01DFFF7E0FE336803EBDD
S31508002E540040306004F10800FFF7D8FE336803EB3E
S31508002E640020306004F10A00FFF7D0FE33681844E6
S31508002E7430600C34053D2DB25FB10026AE4208DA47
S31508002E842046FFF7C3FEB85502340136B6B2F5E755
S31508002E9400252846F8BD4FF0FF35FAE70457000821
S31508002EA4B54B1B78002B00F0F58170B5012B05D0C6
S31508002EB4022B30D0032B00F0208170BDFFF76CFC89
S31508002EC4FDF7C0F9AD48FDF701FAAD48FDF7FEF97F
S31508002ED4FDF7B4F901220146AA4801F035FE48B1C6
S31508002EE4A54B00221A70A848FDF7F0F90120FDF752
S31508002EF4DFF9E2E7A548FDF7E9F9A548FDF7E6F99C
S31508002F04A448FDF7E3F9A44B00221A605A609A4BC9
S31508002F1402221A70D1E7A14C04F50C724FF48071A1
S31508002F249F4802F033FA94F84132002B5DD1A8B1D8
S31508002F349B48002200F5C071FFF716FF0446B0F15E
S31508002F44FF3F60D0002809DD934B5B68002B67D1EF
S31508002F54934BD3F88021904B1A6058608F4BD3F863
S31508002F644422D3F83C329A42A7D10021854802F07C
S31508002F74CBF8002840F0A780874B5B6873B3834877
S31508002F84FDF7A4F98748FDF7A1F9874D824C294630
S31508002F946068FFF7F7FD2846FDF798F98348FDF7BB
S31508002FA495F92946E078FFF721FEA91CA078FFF7D2
S31508002FB41DFE291D6078FFF719FEA91D2078FFF765
S31508002FC415FE2846FDF782F97948FDF77FF9616809
S31508002FD42068FFF7E9FB002800F082806B48FDF7BC
S31508002FE475F9654B03221A7067E7634B00221A705A
S31508002FF46548FDF76BF90220FDF75AF904F50C70DC
S3150800300402F06EF859E75C4B00221A705E48FDF729
S315080030145DF90320FDF74CF95A4802F061F84CE7CC
S315080030245F4AD2F880115C4A12681A44914203D165
S315080030340344594A536091E75448FDF747F95948F8
S31508003044FDF744F9584E544D31466868FFF79AFD22
S315080030543046FDF73BF95548FDF738F93146E87827
S31508003064FFF7C4FDB11CA878FFF7C0FD311D6878C9
S31508003074FFF7BCFDB11D2878FFF7B8FD3046FDF70C
S3150800308425F94B48FDF722F969682868FFF78CFB90
S3150800309460B13E48FDF71AF93E48FDF717F9404B6B
S315080030A4D3F880213C4B1A605C6057E7324B002208
S315080030B41A703548FDF70AF90520FDF7F9F831487D
S315080030C402F00EF8F9E62C4B00221A702E48FDF78A
S315080030D4FDF80420FDF7ECF82A4802F001F8ECE6BE
S315080030E4254B00221A702848FDF7F0F80520FDF74D
S315080030F4DFF8244801F0F4FFDFE6284C04F50C72E7
S315080031044FF48071264802F041F994F84132002BB5
S3150800311456D160B1224800F5807200F5C071FFF7F8
S3150800312423FE0446B0F1FF3F58D0002863DC1B4B4E
S31508003134D3F84422D3F83C329A427FF4BEAE1D48F3
S31508003144FDF7C4F8FFF73CFB002800F096800F480B
S31508003154FDF7BCF81848FDF7B9F80A4801F0C0FFAE
S315080031641648FDF7B3F8044B00221A70FDF77EF8EB
S31508003174FFF71AF9A1E600BF5C0D002034570008D2
S3150800318458570008340B0020805700088857000851
S3150800319490570008B4570008FC08002004090020CA
S315080031A4600D0020E4570008E40E0020F0570008DC
S315080031B4945800087C58000898580008B058000825
S315080031C4354B00221A703548FDF780F80220FDF7C2
S315080031D46FF804F50C7001F083FF6EE62E4B00229F
S315080031E41A702F48FDF772F80320FDF761F82D4889
S315080031F401F076FF61E62C48FDF768F82B4D294661
S315080032042046FFF7BFFC2846FDF760F82848FDF777
S315080032145DF8284E294696F88301FFF7E7FCA91CB2
S3150800322496F88201FFF7E2FC291D96F88101FFF75B
S31508003234DDFCA91D96F88001FFF7D8FC2846FDF7A2
S3150800324445F81D48FDF742F806F580722146D6F87A
S315080032548001FFF7A5FA18B11848FDF737F866E7AD
S315080032640D4B00221A701648FDF730F80620FDF7B4
S315080032741FF80C4801F034FF1FE6074B00221A70AA
S315080032840F48FDF723F80720FDF712F8054801F063
S3150800329427FF12E6704700BF5C0D00200C58000893
S315080032A430580008340B002054580008E40E002057
S315080032B464580008600D00209458000888570008D0
S315080032C480570008014B00225A707047240F0020CB
S315080032D4034BFE22DA7018710222A3F844207047C1
S315080032E4240F002010B5054C00232370FFF7EAFFCE
S315080032F4FF23E3700123A4F8443010BD240F0020F3
S31508003304064BFF22DA7000221A71597859719A719C
S31508003314DA711A720622A3F844207047240F002093
S3150800332408B50020FFF7D4FF08BD0000074BFF22AD
S31508003334DA70074A9A6400221A715A719A71072236
S31508003344C3F807200822A3F844207047240F002056
S31508003354DC580008044BFF22DA7042689A6401229A
S31508003364A3F84420704700BF240F002008B5312075
S31508003374FFF7AEFF08BD000038B5084CFF23E3701D
S31508003384002525716571FFF7C9FBA071E5712572E2
S3150800339465720723A4F8443038BD00BF240F002003
S315080033A438B5FFF779FCE8B1FFF78CFF0F4C012518
S315080033B42570FF23E3701023237100236371FFF73D
S315080033C4ADFBA071FFF7BCFBE071FFF7B9FBC0F3D7
S315080033D4072020726572A5720823A4F84430FFF703
S315080033E4DBF938BD1020FFF773FFFAE7240F002036
S315080033F438B505464478FFF791FB0138844210DC5A
S315080034040A4C6A78A16C201DFEF7EEFFFF23E370D1
S315080034146A78A36C1344A3646B780133A4F8443024
S3150800342438BD2220FFF754FFFAE700BF240F002017
S3150800343438B504464578FFF771FB0138854211DC37
S3150800344461680A4DA9646278281DFEF7CDFFFF233B
S31508003454EB706278AB6C1344AB6463780133A5F8FC
S31508003464443038BD2220FFF733FFFAE7240F002043
S31508003474F8B505461746002406E015F8013B1C4432
S31508003484E4B2FFF77BFB31464E1E0029F5D13C60BA
S315080034940120F8BD10B5084CFF23E370E21D41680E
S315080034A4A06CFFF7E5FF207100236371A37108235D
S315080034B4A4F8443010BD00BF240F002038B50546D3
S315080034C40D4B9C6CFFF72AFB6A1C411E2046FFF72E
S315080034D467F960B1084CFF23E370FFF71FFB013857
S315080034E4A36C0344A3640123A4F8443038BD3120F3
S315080034F4FFF7EEFEFAE700BF240F002038B50446AE
S315080035044578FFF70BFB023885420EDC114BFF2288
S31508003514DA700122A3F84420617851B9FFF750F90B
S3150800352430B93120FFF7D4FE02E02220FFF7D0FE9F
S3150800353438BDA21C074B986CFFF732F928B161789D
S31508003544044A936C0B449364F2E73120FFF7C0FEF8
S31508003554EEE700BF240F002008B54168074B986CB6
S31508003564FFF722F930B1054BFF22DA700122A3F8DE
S31508003574442008BD3120FFF7ABFEFAE7240F0020EC
S3150800358408B5FEF711FF034BFF22DA700122A3F8F0
S31508003594442008BD240F002008B589B2FFF7A6FA0F
S315080035A408BD0000054B00221A709A6483F843206C
S315080035B4A3F844209A705A70704700BF240F00205D
S315080035C4034B1B780BB1012070470020704700BFDE
S315080035D4240F0020024B002283F84320704700BFC3
S315080035E4240F002008B50378FF2B04D0354A127837
S315080035F4012A14D008BDFFF7D3FE324B93F84330A3
S31508003604012B5AD02F4BB3F944100029F2DD184682
S31508003614012380F843300330FFF7BEFFEAE7C93BCE
S31508003624352B46D8DFE803F03345454245453F3652
S315080036343C3945454545454545454545454545453D
S315080036444545454545454545454545454545454518
S315080036544545241E1B2145454527452A2D30FFF798
S31508003664C7FECAE7FFF7E4FEC7E7FFF773FEC4E73A
S31508003674FFF710FFC1E7FFF759FEBEE7FFF750FE55
S31508003684BBE7FFF73DFEB8E7FFF72CFEB5E7FFF704
S3150800369415FFB2E7FFF732FFAFE7FFF76DFEACE7BA
S315080036A4FFF75AFFA9E7FFF76BFFA6E7FFF75EFEEA
S315080036B4A3E72020FFF70CFE9FE71020FFF708FE7C
S315080036C4A0E700BF240F00204278007840EA0220D1
S315080036D47047C278837843EA0222437843EA02238E
S315080036E4007840EA032070470170090A4170704760
S315080036F40170C1F307234370C1F307438370090EAE
S31508003704C170704713462AB10A7802700130013134
S31508003714013BF9D1704701700130013AFBD170477A
S3150800372430B4451C037808781B1A013A04D04C1C9B
S3150800373428462146002BF4D0184630BC704700E0D2
S31508003744013003780BB18B42FAD118467047023917
S315080037544369023B8B4204D94389806A01FB03000F
S3150800376470470020704770B506460D4601F11A00E9
S31508003774FFF7AAFF3378032B00D070BD044605F182
S315080037841400FFF7A1FF44EA0040F6E770B50646C1
S315080037940C46154691B204F11A00FFF7A5FF3378D3
S315080037A4032B00D070BD290C04F11400FFF79CFF0D
S315080037B4F8E700002DE9F04107460E4601F11A0024
S315080037C4FFF782FF60BB357805F03F05013D05EB41
S315080037D4450305EB83054FF00108002404E04FF682
S315080037E4FF73984221D101340C2C0ED8124B185D64
S315080037F43044FFF769FFB8F1000FF0D0FE2D12D858
S3150800380427F8150080460135EDE7337813F0400FA5
S315080038140DD0FE2D0DD8002327F81530012000E021
S315080038240020BDE8F0810020FBE70020F9E701202D
S31508003834F7E70020F5E700BF645900082DE9F843C7
S3150800384480460F4691464B730F23CB7200240C73A4
S31508003854214607F11A00FFF747FF09F1FF3606EB81
S31508003864460306EB8306254602E001340C2C11D8E0
S315080038744FF6FF739D4202D038F8165001360C4BAA
S31508003884185D29463844FFF72FFF002DEDD14FF672
S31508003894FF75EAE74FF6FF739D4202D038F81630F3
S315080038A40BB949F0400987F80090BDE8F88300BFD2
S315080038B46459000870B582B0054616461C460B22A4
S315080038C4FFF720FF052C11D807221DE001320F2A25
S315080038D40CD803F0010101EB44045B0814F4803F9F
S315080038E4F4D084F4883484F02104EFE73388002B79
S315080038F4EAD002360022EAE7531E02A8024402F876
S31508003904081C240909D01A4604F00F0303F13001F0
S315080039143929F1D903F13701EEE77E2102461A4423
S3150800392402F8081C00E001349C4209D22A5D202AC8
S31508003934F9D105E02021621C2955072A08D814461E
S31508003944072BF7D802AA1A4412F8081C0133F2E71F
S3150800395402B070BD01460B220020C30143EA50039E
S31508003964DBB208780344D8B20131013AF5D170477D
S31508003974016809B10A4603E04FF0FF3308E0013253
S3150800398413781F2B01D93A2BF9D13A2B02D00023ED
S315080039941846704710B44C1C0B78303B092B07D8D3
S315080039A4A24208D153B901320260184610BC7047C6
S315080039B44FF0FF33F9E74FF0FF33F6E74FF0FF33E5
S315080039C4F3E738B50D4640B1044603682BB11A78B7
S315080039D41AB1D9888288914203D000232B60092022
S315080039E438BD5878FEF726FA10F0010FF5D123688A
S315080039F42B600020F4E7F8B5C3780BB90020F8BDAE
S31508003A040446C56A00F1300701232A463946407838
S31508003A14FEF762FAA8B90023E370236AEB1AA269CF
S31508003A24934210D2A678012E09D9A3691D4401230D
S31508003A342A4639466078FEF74FFA013EF3E7002036
S31508003A44DDE70120DBE70020D9E770B5C36A8B42BE
S31508003A5412D004460D46FFF7CEFF064668B9012381
S31508003A642A4604F130016078FEF7EEF910B1012612
S31508003A744FF0FF35E56200E00026304670BD0000D1
S31508003A8410B504460023C3704FF0FF33C362FFF733
S31508003A94DCFFD8B904F22E20FFF716FE4AF65523A2
S31508003AA4984215D104F16600FFF713FE20F07F4013
S31508003AB40A4B98420ED004F18200FFF70AFE20F062
S31508003AC47F40064B984207D1002002E0042000E01C
S31508003AD4032010BD0020FCE70220FAE74641540003
S31508003AE42DE9F04784B00F46164600230B60FFF70E
S31508003AF43FFF051EC0F24181B54B53F82540002C03
S31508003B0400F03F813C6006F0FE06237873B16078C6
S31508003B14FEF790F910F0010F08D1002E00F033815A
S31508003B2410F0040F40F03181002027E100232370B0
S31508003B34E8B26070FEF7D6F810F0010F40F027815E
S31508003B441EB110F0040F40F0248100212046FFF72F
S31508003B5497FF022800F0B3800026042800F01B8192
S31508003B64012800F21A8104F13B00FFF7ADFDB0F518
S31508003B74007F40F0148104F14600FFF7A5FD0746CF
S31508003B8420B904F15400FFF7A4FD0746A76194F889
S31508003B944020A270531EDBB2012B00F2028107FB00
S31508003BA402F594F83D80A4F80A80B8F1000F00F0F5
S31508003BB4FA8008F1FF3318EA030F40F0F68004F19F
S31508003BC44100FFF781FD8246208110F00F0F40F077
S31508003BD4EE8004F14300FFF777FD814620B904F12E
S31508003BE45000FFF776FD814604F13E00FFF76CFDB1
S31508003BF40146002800F0DD80421902EB1A129145AD
S31508003C04C0F0D980A9EB0203B3FBF8F3002B00F04C
S31508003C14D48040F6F570834269D84FF001094FF60F
S31508003C24F570834201D94FF0030903F10208C4F879
S31508003C341480E6618B1923623244A262B9F1030F38
S31508003C4458D0BAF1000F00F0BE802B446362B9F174
S31508003C54020F60D008EB480208F0010303EB520395
S31508003C6403F2FF13B7EB532FC0F0AF804FF0FF33C7
S31508003C742361E36080232371B9F1030F4ED084F8DE
S31508003C840090544A138801339BB21380E3800020C2
S31508003C9474E0002004AB03EB850343F8100C0135EC
S31508003CA4032D0ED804F130002B0103F5DF731844F5
S31508003CB40379002BEDD00830FFF70BFDEAE7002562
S31508003CC4EEE700250AE031462046FFF7D9FE01282B
S31508003CD47FF643AF0135032D3FF63FAF04AB03EB45
S31508003CE4850353F8106C002EEDD10320F2E74FF04C
S31508003CF4020994E704F15A00FFF7E6FC00285ED1AE
S31508003D04BAF1000F5DD104F15C00FFF7E2FC6062D2
S31508003D144FEA8803A4E74FEA4803A1E704F16000E1
S31508003D24FFF7D2FC0128AAD1711C2046FFF78DFEA5
S31508003D340028A4D10023237104F22E20FFF7C4FC23
S31508003D444AF6552398429AD104F13000FFF7C1FC8C
S31508003D54214B984293D104F50570FFF7BAFC1F4B23
S31508003D6498428CD104F50670FFF7B3FC206104F57C
S31508003D740770FFF7AEFCE06081E70B2004B0BDE8EE
S31508003D84F0870C20FAE70020F8E70A20F6E7032074
S31508003D94F4E70A20F2E70120F0E70D20EEE70D200C
S31508003DA4ECE70D20EAE70D20E8E70D20E6E70D200D
S31508003DB4E4E70D20E2E70D20E0E70D20DEE70D201D
S31508003DC4DCE70D20DAE70D20D8E70D20D6E700BF9B
S31508003DD4700F0020740F00205252614172724161C3
S31508003DE4F8B50668012952D973698B4251D90C462C
S31508003DF43378022B2BD0032B38D0012B01D001208A
S31508003E0446E001EB5105316A01EB55213046FFF7CF
S31508003E141CFE00283FD16F1CC5F30805354495F8E8
S31508003E243050316A01EB57213046FFF70EFEA8BB26
S31508003E34C7F308073E4496F8300045EA002014F014
S31508003E44010F01D0000923E0C0F30B0020E0316A1A
S31508003E5401EB14213046FFF7F8FD10BB600000F4AF
S31508003E64FF7030303044FFF72FFC11E0316A01EB64
S31508003E74D4113046FFF7E9FDB0B9A00000F4FE708E
S31508003E8430303044FFF725FC20F0704000E0012074
S31508003E94F8BD0120FCE74FF0FF30F9E74FF0FF309B
S31508003EA4F6E74FF0FF30F3E74FF0FF30F0E72DE980
S31508003EB4F0410768B1F5001F3BD206460D4611F0DE
S31508003EC41F0F39D1316184681CB93B78022B00D99C
S31508003ED47C6A94B93B89B3EB551F2FD97B6AB361C6
S31508003EE47461B36993B303EB5523B3613037C5F3F0
S31508003EF408053D44F56100201CE0B7F80A804FEA3E
S31508003F04482845450FD321463046FFF769FF04463E
S31508003F14B0F1FF3F14D0012814D97B69834213D921
S31508003F24A5EB0805EDE721463846FFF710FCB06116
S31508003F34D6E70220BDE8F0810220FBE70220F9E774
S31508003F440120F7E70220F5E70220F3E70220F1E76C
S31508003F542DE9F84301297CD943698B427BD9164656
S31508003F640C4605460378022B47D0032B57D0012B62
S31508003F7401D0022770E001EB5108016A01EB5821D0
S31508003F84FFF763FD0746002866D108F10109C8F35F
S31508003F94080814F0010423D005EB080393F930301C
S31508003FA403F00F03320102F47F621343DBB2A84421
S31508003FB488F830300123EB70296A01EB5921284629
S31508003FC4FFF743FD0746002846D1C9F308094CB153
S31508003FD4C6F30712A94489F830200123EB703BE0A5
S31508003FE4F3B2E4E705EB090393F9302022F00F0254
S31508003FF4C6F303263243D2B2ECE7016A01EB142175
S31508004004FFF723FD074638BB600000F4FF70303025
S31508004014B1B22844FFF768FB0123EB701CE0016A80
S3150800402401EBD411FFF711FD0746A8B926F070462F
S31508004034A40004F4FE7430342C442046FFF749FBEC
S3150800404400F0704131432046FFF752FB0123EB7021
S3150800405402E0022700E002273846BDE8F8832DE986
S31508004064F04107460668884631B9F5688DB1736923
S31508004074AB420FD801250DE0FFF7B2FE034601282F
S3150800408447D9B0F1FF3F49D07269824246D84546BE
S3150800409400E001252C460CE021463846FFF7A0FE31
S315080040A4034670B1012839D0B0F1FF3F36D0AC428F
S315080040B433D001347369A342EED8012D2BD90224D7
S315080040C4EAE74FF0FF3221463046FFF741FF034641
S315080040D410B9B8F1000F0ED1A3B9F4603269736947
S315080040E4023B9A4201D2013A3261337943F0010321
S315080040F43371234612E0224641463046FFF728FF2D
S315080041040346E9E7012B01D0012307E04FF0FF330B
S3150800411404E0012302E0002300E000231846BDE87A
S31508004124F081F8B50E46046801292ED907461146CA
S315080041346369B3422BD95AB14FF0FF322046FFF7D1
S3150800414407FF024620B123E063692E46AB421FD916
S3150800415431463846FFF744FE0546D8B101281BD038
S31508004164B0F1FF3F1AD0002231462046FFF7F0FE91
S31508004174024668B92369B3F1FF3FE5D001332361E9
S31508004184237943F001032371DEE7022200E00222C9
S315080041941046F8BD0022FBE70222F9E70122F7E7F9
S315080041A42DE9F843066805698369002B6DD0203527
S315080041B4B5F5001F6BD288460446C5F308073FB910
S315080041C401338361416971B93389B3EB551F06D944
S315080041D4256130373E44E6610020BDE8F8830023B4
S315080041E483610420F9E77389013B13EA5523EFD168
S315080041F4FFF7F6FD814601284BD9B0F1FF3F4AD0B7
S315080042047369834239D8B8F1000F11D06169204621
S31508004214FFF725FF814600283FD001283FD0B0F19B
S31508004224FF3F3ED03046FFF7E6FB28B10120D4E72E
S315080042340023A3610420D0E74FF40072002106F19D
S315080042443000FFF768FA49463046FFF780FAF0620D
S315080042544FF00008738998450BD20123F370304652
S31508004264FFF7C9FBF8B908F10108F36A0133F362E9
S31508004274F0E7F36AA3EB0803F362C4F8149049461B
S315080042843046FFF764FAA061A2E70420A5E70420F4
S31508004294A3E70220A1E701209FE707209DE7022064
S315080042A49BE7012099E7012097E7F8B504460F46EE
S315080042B406680021FFF7FBFD0346C0B9002508E0A0
S315080042C40135BD4213D001212046FFF769FF034695
S315080042D468B9A1693046FFF7B8FB034638B9E269FD
S315080042E41278E52AECD0002AEAD00025EBE7042B5D
S315080042F401D01846F8BD0723FBE72DE9F843044621
S31508004304884607684FF0FF094E4604252EE00F2B12
S3150800431419D112F0400F06D091F80D9002F0BF02A1
S31508004324236963621646B24201D0FF2618E04B7B26
S315080043344B4501D0FF2613E0A06AFFF73BFA88B382
S31508004344013EF6B20CE026B90846FFF703FB4845DA
S315080043542BD04FF0FF33636227E0FF2600E0FF26E9
S3150800436400212046FFF71CFF0546F0B9A169E1B113
S315080043743846FFF76AFB0546B8B9E1690A789AB17F
S31508004384CB7A03F03F03A371E52AE6D02E2AE6D0BA
S3150800439423F02000082814BF002001204045B6D089
S315080043A4FF26DDE7FF26DBE704250DB10023A3611D
S315080043B42846BDE8F88370B5044605680669416A67
S315080043C4B1F1FF3F18D1A1692846FFF73EFB034622
S315080043D470B9E269E52111700122EA702269B242D4
S315080043E406D200212046FFF7DBFE03460028EAD062
S315080043F4042B07D0184670BDFFF759FD034600285D
S31508004404E1D0F7E70223F5E72DE9F04F83B08046BC
S315080044148A46D1F80090856A002411E0013609EB32
S31508004424060219F806302F2BF8D05C2BF6D0CAF8FA
S3150800443400201F2821D8042722E025F814703446C2
S31508004444661C19F804001F28E9D92F28E7D05C2828
S31508004454E5D0FE2C00F2DF80012100F0E9FF0746D3
S31508004464002800F0DA807F28E7D801466D48FFF770
S3150800447466F90028E1D0062086E0002700E0013C22
S3150800448444B104F10043013B35F81330202BF6D030
S315080044942E2BF4D0002325F81430002C00F0BF800E
S315080044A40B222021D8F82000FFF735F9002300E075
S315080044B4013335F81320202AFAD02E2AF8D01BB156
S315080044C447F0030700E0013C6CB104F10042013AED
S315080044D435F812202E2AF6D14FF0080B4FF0000AB1
S315080044E4CDF804A00AE0A2464FF0080B0022019278
S315080044F404E04C450BD047F003074B4603F101098A
S3150800450435F81360FEB1202EF5D02E2EF1D0DA45FB
S3150800451410D24C450ED07F2E46D8002E51D147F0E6
S3150800452403075F26D8F8203003F80A604B460AF1D9
S31508004534010AE3E7BBF10B0F29D04C4501D047F03C
S3150800454403074C4526D2D8F820301A78E52A54D0E1
S31508004554BBF1080F54D0019B03F00C020C2A03D0BC
S3150800456403F00303032B01D147F0020717F0020FE8
S3150800457406D1019B03F00303012B46D0042A47D036
S31508004584D8F82030DF72002003B0BDE8F08F47F07A
S315080045940307D8E7019B9B00DBB2019323464FF040
S315080045A40B0B4FF0080AA9E70021304600F040FF3C
S315080045B4064618B1A0F180061B4B9E5D47F002071C
S315080045C4ABE731461948FFF7BAF80028A7D1A6F190
S315080045D441039BB2192B04D8019B43F002030193B0
S315080045E4A0E7A6F161039BB2192B9BD8019B43F064
S315080045F401030193203EB6B294E705221A70A7E791
S31508004604019B9B00DBB20193A5E747F01007B5E7CA
S3150800461447F00807B4E70620B6E70620B4E70620FD
S31508004624B2E700BF74590008E45800088059000826
S31508004634F8B500238B758369002B6BD00D460646A7
S31508004644436AB3F1FF3F13D0836A00249F1C18887A
S3150800465458B1002100F0ECFE30B1FE2C0CD82A1912
S3150800466490753B460134F1E700242C440023A375D6
S31508004674A87D0022134612E00024F6E7E52317E096
S3150800468410B9A9182E278F75A9182E274F7201322B
S3150800469410E010211CE0A9188B75013223460A2B59
S315080046A41BD8F1695C1CCB5C202BF7D0052BE5D015
S315080046B4092CE5D0A9184B720028EED1A3F14101C3
S315080046C4C9B21929E7D8F1690F7B082CE1D8082162
S315080046D40F42E0D02033DBB2DDE730B9AB18002156
S315080046E49975F3691B7B03B90A462A440023537256
S315080046F4F369DB7A2B72F0691C30FEF7EAFF28604F
S31508004704F0691830FEF7E0FFA880F0691630FEF766
S31508004714DBFFE880F8BD00002DE9F04781460F4627
S3150800472401F11A00FEF7D0FFB8BB3D7805F03F0546
S31508004734013D05EB450305EB83054FF0010800240D
S3150800474404E04FF6FF7398422ED101340C2C18D886
S31508004754194B185D3844FEF7B7FF0646B8F1000F43
S31508004764EFD0FE2D1CD800F07FFE804605F1010A25
S3150800477439F8150000F078FE804513D1B046554641
S31508004784E3E73B7813F0400F10D0B8F1000F0FD0D1
S3150800479439F8153073B9012000E00020BDE8F08728
S315080047A40020FBE70020F9E70020F7E70120F5E7FA
S315080047B40120F3E70020F1E7645900082DE9F843DE
S315080047C40446D0F800800021FFF771FB064600284E
S315080047D45ED14FF0FF3363624FF0FF094F460AE09C
S315080047E44FF0FF336362FF2700212046FFF7D8FC0A
S315080047F4064600284CD1A1694046FFF726F9064625
S31508004804002845D1E5692B78002B40D0E97A01F0D8
S315080048143F02A271E52BE3D011F0080F01D00F2A4D
S31508004824DED10F2A14D027B92846FFF793F848454E
S315080048342ED0216ACB7A13F0010F04D10B22284615
S31508004844FEF76EFF20B34FF0FF336362FF27CBE713
S31508004854A06A0028C8D013F0400F06D095F80D902A
S3150800486403F0BF03226962621F46BB4201D0FF27D9
S31508004874BAE76B7B4B4501D0FF27B5E72946FFF717
S315080048844BFF10B1013FFFB2AEE7FF27ACE70426A2
S315080048943046BDE8F88330B583B00446019105680F
S315080048A401E001330193019B1A782F2AF9D05C2A77
S315080048B4F7D00022A2601B781F2B1DD901A9204618
S315080048C4FFF7A2FD0346F8B92046FFF777FF236AE8
S315080048D4DA7A0346D8B912F0040F15D1A37913F07E
S315080048E4100F1BD02169C1F3080130312944284629
S315080048F4FEF739FFA060E1E7236A8022DA72002115
S315080049042046FFF7D4FA0346184603B030BD0428F8
S31508004914FAD112F0040FF7D10523F5E70523F3E7D7
S315080049242DE9F04784B00668D0F820A0D0F828808E
S315080049349AF80B3013F0A00F40F08980002400E0A9
S31508004944013438F81430002BFAD105460C225146A6
S3150800495401A8FEF7D7FE9DF80F3013F0010F1ED0FD
S3150800496400238AF80B30AB620127632F0CD83B4629
S31508004974424601A95046FEF79DFF2846FFF71EFF4B
S31508004984814608B90137F0E7642F66D0B9F1040FF8
S315080049945FD19DF80F308AF80B30C5F828809DF84A
S315080049A40F3013F0020F2AD00C342D4BA3FB04341A
S315080049B4A408013421462846FFF777FC814608B93E
S315080049C4013C1ED1B9F1000F43D1A9693046FFF75E
S315080049D43CF8814600283CD120220021E869FEF7EC
S315080049E49AFE0B22296AE869FEF78CFE2B6ADB7AA3
S315080049F4EA6903F0180313730123F37029E0012409
S31508004A04D8E72969A1EB44112846FFF750FA8146ED
S31508004A140028D7D1286AFEF79DFF0746A9693046BC
S31508004A24FFF713F881460028CCD13B46E2B2E96980
S31508004A34A86AFEF703FF0123F37000212846FFF74F
S31508004A44AFFB81460028BDD1013CE7D1BAE74FF058
S31508004A540609484604B0BDE8F0874FF00709F8E7A9
S31508004A644FECC44E70B50446FEF7C5FF054648B973
S31508004A742378032B08D0002211466078FDF786FABE
S31508004A8400B10125284670BD2379012BF3D104F121
S31508004A9430064FF4007200213046FEF73CFE4AF613
S31508004AA4552104F22E20FEF71FFE0F493046FEF765
S31508004AB41FFE0E4904F50570FEF71AFE216904F572
S31508004AC40670FEF715FEE16804F50770FEF710FE9A
S31508004AD4E2690132E262012331466078FDF7FCF9A6
S31508004AE400232371C7E700BF5252614172724161C4
S31508004AF410B584B001900091144604A840F8041D2A
S31508004B04FEF736FF002819DB0E4B53F820300BB19D
S31508004B1400221A70019B0BB100221A70019B094AE4
S31508004B2442F8203063B1012C02D0002004B010BD35
S31508004B34002201A96846FEF7D3FFF7E70B20F5E73D
S31508004B440020F3E7700F00202DE9F04393B001919C
S31508004B54002800F0AF80044615460023036002F0DF
S31508004B641F073A4606A901A8FEF7BAFF064618B172
S31508004B74304613B0BDE8F083069B079303AB0F9347
S31508004B844D4B1193019907A8FFF785FE064620B9F0
S31508004B940F9B93F90B30002B46DB15F01C0F54D0F2
S31508004BA4002E48D0042E41D047F00807002E5BD1CA
S31508004BB417F0080F58D0414D29460E980E30FEF7C7
S31508004BC497FD29460E981630FEF792FD0E9B202275
S31508004BD4DA72069DDDF8388041462846FEF7C3FD9D
S31508004BE48146002241462846FEF7D0FD00210E984C
S31508004BF41C30FEF77DFD069B0122DA70B9F1000F21
S31508004C0432D0069BDD6A0022494607A8FFF789FACF
S31508004C14064648BB29460698FEF717FF064609F1D5
S31508004C24FF33069AD3601FE00626B6E707A8FFF700
S31508004C3477FE0646B8E79DF8223013F0110F12D115
S31508004C4415F0040FB2D008260EE06EB99DF822308E
S31508004C5413F0100F2CD115F0020F05D013F0010F25
S31508004C6402D007260BE007264EB917F0080F01D025
S31508004C7447F02007069BDB6A23620E9B6362002EBD
S31508004C847FF476AF069DDDF8388041462846FEF760
S31508004C946AFDA06008F11C00FEF71BFDE060002316
S31508004CA463746361E36127742560EB88A3805FE717
S31508004CB40426E4E709265BE7780F0020000061482C
S31508004CC42DE9F04F85B004468946174698460023D1
S31508004CD4C8F8003003A9FEF774FE0646002840F01B
S31508004CE4A280667C002E40F09E80237C13F0010F80
S31508004CF400F0A380E5686369ED1ABD425DD33D46BD
S31508004D045BE0A1692046FFF76BF866E00226667445
S31508004D1489E00126667486E00226667483E0237CAD
S31508004D2413F0400F05D0E069A0EB0A00019B9842F6
S31508004D3402D3019B5F0236E04FF4007204F12801A6
S31508004D4409EB4020FEF7DEFCF3E7E26952451AD088
S31508004D54237C13F0400F0CD0012304F128019BF89F
S31508004D640100FDF7B9F8002861D1237C23F040033C
S31508004D7423740123524604F1280103984078FDF769
S31508004D8463F8002856D1C4F81CA06169C1F3080168
S31508004D94C1F50077BD4200D22F4628313A46214450
S31508004DA44846FEF7AFFCB94463693B446361D8F8E7
S31508004DB400303B44C8F80030ED1B002D33D063693E
S31508004DC4C3F30802002AE0D1039A5789013F17EA78
S31508004DD4532708D1002B94D1A068012896D9B0F19D
S31508004DE4FF3F96D0A061DDF80CB0A1695846FEF7DE
S31508004DF4AEFC824600288FD0BA446B0A0193A4D02D
S31508004E04FB18BBF80A20934201D9D31B0193019BD3
S31508004E14524649469BF80100FDF716F800283FF468
S31508004E247EAF01266674304605B0BDE8F08F0126CC
S31508004E346674F8E701266674F5E70726F3E72DE9AD
S31508004E44F04F85B004468846154699460023C9F8A6
S31508004E54003003A9FEF7B5FD0746002840F0B280E6
S31508004E64677C002F40F0AE80237C13F0020F00F01D
S31508004E74BF806369EB4264D3DD4362E000212046C8
S31508004E84FFF7EDF86FE0A1692046FFF7E8F86AE056
S31508004E940227677496E00127677493E00123E269A1
S31508004EA404F1280103984078FDF716F820B9237C05
S31508004EB423F04003237465E00127677482E0022720
S31508004EC467747FE0E169A1EB0A01594502D34FEA09
S31508004ED44B2627E04FF4007208EB412104F1280021
S31508004EE4FEF710FC237C23F040032374EFE7E36901
S31508004EF4534503D06269E3689A4267D3C4F81CA091
S31508004F046069C0F30800C0F50076B54200D22E46A3
S31508004F142830324641462044FEF7F4FB237C43F00E
S31508004F2440032374B044636933446361E26893427B
S31508004F3438BF1346E360D9F800303344C9F8003063
S31508004F44AD1B002D4FD06369C3F30802002AD7D1DD
S31508004F54039A5689013E16EA53260FD1002B92D19D
S31508004F64A06800288AD000283DD0012890D0B0F146
S31508004F74FF3F90D0A061A36803B9A060237C13F017
S31508004F84400F8BD1039B0193A1691846FEF7DFFBFB
S31508004F948246002893D0B2445FEA552BA7D006EB85
S31508004FA40B03019A5289934201D9A2EB060B5B467D
S31508004FB45246414601984078FCF78EFF002881D076
S31508004FC401276774384605B0BDE8F08F01235246B9
S31508004FD404F1280101984078FCF736FF00288DD0A3
S31508004FE401276774EEE7237C43F020032374E9E77B
S31508004FF40727E7E770B582B004460D460A290DD09F
S315080050046368002B08DB5E1C23441D733C2E09DCF5
S315080050146660A3680133A36002B070BD0D21FFF773
S31508005024E9FFEDE701AB324604F10C012068FFF70E
S3150800503406FF019B9E4202D04FF0FF36E8E70026A2
S31508005044E6E7000030B583B0044601A9FEF7B9FCCB
S315080050540346C8B9227C12F0200F15D012F0400F6F
S315080050640CD00123E26904F1280101984078FCF781
S3150800507433FF88BB237C23F040032374216A0198F9
S31508005084FEF7E3FC034610B1184603B030BD656A63
S31508005094EB7A43F02003EB72A26829462068FEF7F0
S315080050A475FBE16805F11C00FEF722FB0B4905F1C7
S315080050B41600FEF71DFB002105F11200FEF714FB8E
S315080050C4019B0122DA700198FFF7CCFC0346227C87
S315080050D422F020022274D7E70123D5E700006148AD
S315080050E410B582B00446FFF7ADFF034610B1184663
S315080050F402B010BD01A92046FEF763FC034600284A
S31508005104F5D100222260F2E72DE9F04182B0044687
S315080051140F4601A9FEF755FC0646002840F0A28072
S31508005124667C002E40F09E80E368BB4204D2227C53
S3150800513412F0020F00D11F46636900226261002F34
S3150800514465D0019AB2F80A804FEA482873B17A1EE4
S31508005154B2FBF8F2013BB3FBF8F18A4206D3C8F175
S31508005164000213406361FF1AA56902E0A56815B138
S31508005174A56135BB4CE000212046FEF770FF0546C5
S31508005184012804D0B0F1FF3F04D0A060F0E702265E
S31508005194667467E00126667464E029462046FEF7CD
S315080051A41FFE0546B5F1FF3F28D0012D29D9019BDD
S315080051B45B69AB4225D9A561636943446361A7EB7F
S315080051C4080747450BD9237C13F0020FE5D0294677
S315080051D42046FEF744FF05460028E3D1474663699F
S315080051E43B446361C7F30803002B3FD02946019863
S315080051F4FEF7ADFA40B100EB572509E001266674BF
S3150800520430E0022666742DE0022666742AE000253C
S315080052146369C3F30803E3B1E269AA4219D0237C9C
S3150800522413F0400F0BD0012304F1280101984078AC
S31508005234FCF752FEE0B9237C23F0400323740123D0
S315080052442A4604F1280101984078FCF7FDFD90B937
S31508005254E5616369E268934204D9E360237C43F019
S3150800526420032374304602B0BDE8F0810025CFE759
S3150800527401266674F6E701266674F3E730B591B03D
S3150800528401900D46002205A901A8FEF729FC04464B
S3150800529410B1204611B030BD02AB0D930B4B0F93E2
S315080052A4019905A8FFF7F7FA04460028F1D10D9BE2
S315080052B493F90B30002B06DB002DEAD0294605A806
S315080052C4FFF7B6F9E5E70624E3E700BF780F002001
S315080052D4F0B59DB00190022205A901A8FEF700FCCD
S315080052E4059B1193044610B120461DB0F0BD02ABD0
S315080052F41993254B1B93019911A8FFF7CCFA044679
S315080053040028F1D1199B93F90B30002B1EDB9DF86D
S315080053144A5015F0010F2AD1059F18993846FEF709
S3150800532422FA064615F0100F12D0069708900021A7
S3150800533406A8FEF7BCFD044650B9002106A8FEF7E8
S31508005344DCFF0446B0B1042802D103E00026062493
S31508005354002CC9D111A8FFF72EF8044600B95EB986
S31508005364002CC1D10598FFF77DFB0446BCE700264F
S315080053740724EDE70724EBE70022314611A8FEF7D8
S31508005384D0FE0446ECE700BF780F00202DE9F04173
S3150800539482B080460E4617460446002501E022469A
S315080053A41446731EAB4212DD6B46012201A9384628
S315080053B4FFF786FC009B012B09D19DF804300D2BC1
S315080053C4EDD0621C237001350A2BE9D1144600235B
S315080053D423701DB1404602B0BDE8F0810020FAE70B
S315080053E410B594B00446019100230293039303E095
S315080053F4013401A8FFF7FEFD21780029F8D1029AA5
S31508005404002A0CDB6B4604A90198FFF718FD48B976
S31508005414029A009B9A4208D1039814B010BD4FF023
S31508005424FF30FAE74FF0FF30F7E74FF0FF30F4E7C5
S315080054347F2816D931B1FF2812D88038094B33F89A
S315080054441000704700237F2B07D8064A32F813202A
S31508005454824202D001339BB2F5E78033D8B2704753
S315080054640020704788590008B0F5805F07D2234B9F
S315080054741A88002A40D090423ED3F0B406E0204B66
S31508005484F6E72B461A88CAB1904217D31D1D5B88C6
S31508005494190ADBB29C18A04204DB0029F1D105EBFA
S315080054A44303EFE7082909D8DFE801F0050A1013D2
S315080054B416191C1F2200861A35F81600F0BC704708
S315080054C4821A02F00103C01A80B2F7E7103880B2D4
S315080054D4F4E7203880B2F1E7303880B2EEE71A38BC
S315080054E480B2EBE7083080B2E8E7503880B2E5E7E7
S315080054F4A0F5E35080B2E1E7704700BF885A000878
S315080055047C5C000870B500250C4E0D4CA41BA41039
S31508005514A54209D100F050F800250A4E0A4CA41BEE
S31508005524A410A54205D170BD56F825309847013513
S31508005534EEE756F8253098470135F2E7445E000849
S31508005544445E0008445E0008485E0008044B054AA9
S315080055541B681B6A002B08BF1346D3F8EC00704778
S31508005564100000207400002082B001B901A942B1DC
S315080055744BB113780B601278101C18BF012002B0C7
S3150800558470471046FBE76FF00100F8E7034602444C
S31508005594934200D1704703F8011BF9E749B1FF2A82
S315080055A48BBF8A230A700360012088BF4FF0FF303F
S315080055B47047084670470000F8B500BFF8BC08BC39
S315080055C49E467047F8B500BFF8BC08BC9E467047AF
S315080055D42F626F6F746C6F672E7478740000000006
S315080055E42F64656D6F70726F675F73746D3332669F
S315080055F43230372E73726563000000000000000025
S315080056040000000001020304060708090000000060
S3150800561401020304433A2F576F726B2F736F667434
S31508005624776172652F4F70656E424C542F546172C0
S315080056346765742F536F757263652F41524D434DD9
S31508005644335F53544D333246322F63616E2E6300F3
S3150800565405020602060307030803090309040A04E4
S315080056640B040C040C050D050E050F050F06100694
S31508005674100710080080000800400000020000001F
S3150800568400C00008004000000300000000000108F4
S3150800569400000100040000000000020800000200E7
S315080056A405000000000004080000020006000000CF
S315080056B4000006080000020007000000433A2F57BE
S315080056C46F726B2F736F6674776172652F4F70658F
S315080056D46E424C542F5461726765742F536F7572FA
S315080056E463652F41524D434D335F53544D33324610
S315080056F4322F72733233322E63000000303A0000C0
S31508005704433A2F576F726B2F736F6674776172659E
S315080057142F4F70656E424C542F5461726765742F0F
S31508005724536F757263652F66696C652E6300000096
S315080057344669726D77617265207570646174652057
S3150800574472657175657374206465746563746564DC
S315080057540A0D00004F70656E696E67206669726D82
S31508005764776172652066696C6520666F722072655A
S315080057746164696E672E2E2E000000004552524F52
S31508005784520A0D004F4B0A0D000000005374617253
S3150800579474696E67207468652070726F6772616DCC
S315080057A46D696E672073657175656E63650A0D00AC
S315080057B450617273696E67206669726D7761726586
S315080057C42066696C6520746F20646574656374204B
S315080057D4657261736520626C6F636B732E2E2E007F
S315080057E445726173696E672000000000206279744F
S315080057F465732066726F6D206D656D6F72792061B1
S31508005804742030780000000052656164696E672070
S315080058146C696E652066726F6D2066696C652E2EDE
S315080058242E4552524F520A0D00000000496E766109
S315080058346C696420636865636B73756D20666F7540
S315080058446E642E2E2E4552524F520A0D0000000049
S3150800585450726F6772616D6D696E67200000000093
S3150800586420627974657320746F206D656D6F727923
S31508005874206174203078000057726974696E672055
S3150800588470726F6772616D20636865636B73756D9B
S315080058942E2E2E00436C6F73696E67206669726DCF
S315080058A4776172652066696C650A0D004669726DD2
S315080058B477617265207570646174652073756363B6
S315080058C465737366756C6C7920636F6D706C65743B
S315080058D465640A0D000000004F70656E424C540062
S315080058E4809A45418E418F804545454949498E8F61
S315080058F49092924F994F555559999A9B9C9D9E9F64
S3150800590441494F55A5A5A6A7A8A9AAABACADAEAF64
S31508005914B0B1B2B3B4B5B6B7B8B9BABBBCBDBEBFFD
S31508005924C0C1C2C3C4C5C6C7C8C9CACBCCCDCECFED
S31508005934D0D1D2D3D4D5D6D7D8D9DADBDCDDDEDFDD
S31508005944E0E1E2E3E4E5E6E7E8E9EAEBECEDEEEFCD
S31508005954F0F1F2F3F4F5F6F7F8F9FAFBFCFDFEFFBD
S3150800596401030507090E10121416181C1E00000060
S31508005974222A3A3C3E3F7C7F000000002B2C3B3D0C
S315080059845B5D0000C700FC00E900E200E400E000FB
S31508005994E500E700EA00EB00E800EF00EE00EC00A3
S315080059A4C400C500C900E600C600F400F600F2000B
S315080059B4FB00F900FF00D600DC00A200A300A50046
S315080059C4A7209201E100ED00F300FA00F100D100EE
S315080059D4AA00BA00BF001023AC00BD00BC00A10099
S315080059E4AB00BB0091259225932502252425612524
S315080059F46225562555256325512557255D255C259C
S31508005A045B251025142534252C251C2500253C2525
S31508005A145E255F255A255425692566256025502562
S31508005A246C25672568256425652559255825522535
S31508005A3453256B256A2518250C25882584258C2548
S31508005A4490258025B103DF009303C003A303C30392
S31508005A54B500C403A6039803A903B4031E22C60308
S31508005A64B50329226122B100652264222023212359
S31508005A74F7004822B0001922B7001A227F20B20084
S31508005A84A025A00061001A03E0001703F800070325
S31508005A94FF000100780100013001320106013901D5
S31508005AA410014A012E017901060180014D004302C5
S31508005AB481018201820184018401860187018701AB
S31508005AC489018A018B018B018D018E018F01900159
S31508005AD49101910193019401F601960197019801A8
S31508005AE498013D029B019C019D0120029F01A00192
S31508005AF4A001A201A201A401A401A601A701A7016C
S31508005B04A901AA01AB01AC01AC01AE01AF01AF0119
S31508005B14B101B201B301B301B501B501B701B801C9
S31508005B24B801BA01BB01BC01BC01BE01F701C00141
S31508005B34C101C201C301C401C501C401C701C80129
S31508005B44C701CA01CB01CA01CD011001DD0101005B
S31508005B548E01DE011201F3010300F101F401F401DF
S31508005B64F8012801220212013A020900652C3B02B7
S31508005B743B023D02662C3F024002410241024602B4
S31508005B840A015302400081018601550289018A01EE
S31508005B9458028F015A0290015C025D025E025F029E
S31508005BA49301610262029401640265026602670255
S31508005BB4970196016A02622C6C026D026E029C01C0
S31508005BC4700271029D01730274029F0176027702C4
S31508005BD4780279027A027B027C02642C7E027F02B6
S31508005BE4A60181028202A90184028502860287022D
S31508005BF4AE014402B101B20145028D028E028F0242
S31508005C0490029102B7017B030300FD03FE03FF0321
S31508005C14AC0304008603880389038A03B1031103CA
S31508005C24C2030200A303A303C4030803CC030300AB
S31508005C348C038E038F03D8031801F2030A00F903B1
S31508005C44F303F403F503F603F703F703F903FA0377
S31508005C54FA033004200350041007600422018A045E
S31508005C643601C1040E01CF040100C004D004440166
S31508005C7461052604000000007D1D0100632C001E3A
S31508005C849601A01E5A01001F0806101F0606201FAB
S31508005C940806301F0806401F0606511F0700591F2D
S31508005CA4521F5B1F541F5D1F561F5F1F601F080688
S31508005CB4701F0E00BA1FBB1FC81FC91FCA1FCB1FE0
S31508005CC4DA1FDB1FF81FF91FEA1FEB1FFA1FFB1F5A
S31508005CD4801F0806901F0806A01F0806B01F0400A8
S31508005CE4B81FB91FB21FBC1FCC1F0100C31FD01F8A
S31508005CF40206E01F0206E51F0100EC1FF21F010061
S31508005D04FC1F4E210100322170211002842101005A
S31508005D148321D0241A05302C2F04602C0201672C09
S31508005D240601752C0201802C6401002D260841FF0A
S31508005D341A0300004300504F534958002E00002010
S31508005D442020202020202020282828282820202019
S31508005D5420202020202020202020202020202088C9
S31508005D64101010101010101010101010101010042D
S31508005D74040404040404040404101010101010107D
S31508005D844141414141410101010101010101010171
S31508005D940101010101010101010110101010101087
S31508005DA44242424242420202020202020202020241
S31508005DB4020202020202020202021010101020005D
S31508005DC400000000000000000000000000000000C1
S31508005DD400000000000000000000000000000000B1
S31508005DE400000000000000000000000000000000A1
S31508005DF40000000000000000000000000000000091
S31508005E040000000000000000000000000000000080
S31508005E140000000000000000000000000000000070
S31508005E240000000000000000000000000000000060
S31508005E340000000000000000000000000000000050
S30908005E44A90100089A
S30908005E4885010008BA
S31508005E4C0024F4000100000010000000010400000A
S31508005E5C14000020000000000000000000000000F4
S31508005E6C0000000000000000000000000000000018
S31508005E7C0000000000000000000000000000000008
S31508005E8C00000000000000000000000000000000F8
S31508005E9C00000000000000000000000000000000E8
S31508005EAC00000000000000000000000000000000D8
S31508005EBC0000000043000000000000000000000085
S31508005ECC00000000000000000000000000000000B8
S31508005EDC0000000043000000000000000000000065
S31508005EEC0000000000000000000000000000000098
S31508005EFC0000000043000000000000000000000045
S31508005F0C0000000000000000000000000000000077
S31508005F1C0000000043000000000000000000000024
S31508005F2C0000000000000000000000000000000057
S31508005F3C0000000043000000000000000000000004
S31508005F4C0000000000000000000000000000000037
S31508005F5C00000000430000000000000000000000E4
S31508005F6C0000000000000000000000000000000017
S31508005F7C00000000430000000000000000000000C4
S31508005F8C00000000000000000000000000000000F7
S31508005F9C00000000A15500086D550008000000001F
S31508005FAC425D0008405D0008415D0008415D00083F
S31508005FBC415D0008415D0008415D0008415D00082F
S31508005FCC415D0008415D0008415D0008FFFFFFFFC9
S31508005FDCFFFFFFFFFFFFFFFFFFFF0000010041531C
S31508005FEC43494900000000000000000000000000C2
S31508005FFC00000000000000000000000000004153F3
S3150800600C43494900000000000000000000000000A1
S3150800601C0000000000000000000000000000000066
S70508000741AA
